:02000000EA29EB
:08000800FF00030E8312031335
:10001000B4000A0EB500040EB6008A110A12122AA4
:10002000CE08031D14280800F930FF3E031D1528D3
:100030000000CE0B14280800D301D101D201D2193F
:1000400008000310D10DCF0DD30D50085302031C2F
:100050002B28D3005114D20A1F28D101D301D20179
:10006000D21908000310D30DCF0DD10D5008510245
:10007000031C3C28D1005314D20A302883120313E6
:10008000BB08BC08BB0A0319BC0A3B08E83ABC1F02
:10009000033003193C06031D08004C0ACC00BB01C9
:1000A000BC014C083B3C03180800CC014A0ACA00BA
:1000B0004A083B3C031808004B0ACB00CA014B0816
:1000C000173C03180800CB01CA01CC0108008312B9
:1000D0000313B908BA08B90A0319BA0A0530390670
:1000E00003193A08031D7828470AC700B901BA0165
:1000F0004708013A03198F28033A0319A228013A45
:100100000319AD28073A0319C028013A0319CB286F
:10011000033A0319DE28013A0319E928FB28C03005
:10012000831606058600C03083120605CF00013015
:100130004F0486004C08CF000A30D0001C20530822
:10014000C800FB28C030831606058600C030831225
:10015000060586000F30C800FB28C0308316060550
:100160008600C03083120605CF0002304F0486009F
:100170004C08CF000A30D0002D205308C800FB28BF
:10018000C030831606058600C0308312060586003F
:100190000F30C800FB28C030831606058600C0302B
:1001A00083120605CF0004304F0486004A08CF00B2
:1001B0000A30D0001C205308C800FB28C03083162A
:1001C00006058600C0308312060586000F30C80081
:1001D000FB28C030831606058600C0308312060552
:1001E000CF0008304F0486004A08CF000A30D00004
:1001F0002D205308C8004708083A03190F29013A6F
:1002000003191A29033A03192D29013A0319382928
:10021000073A03194B29013A031956295829C030C6
:10022000831606058600C0308312060586000F304F
:10023000C8005829C030831606058600C0308312D6
:100240000605CF0010304F0486004B08CF000A305F
:10025000D0001C205308C8005829C030831606055A
:100260008600C0308312060586000F30C80058296A
:10027000C030831606058600C03083120605CF0005
:1002800020304F0486004B08CF000A30D0002D20CC
:100290005308C8005829C030831606058600C030B0
:1002A0008312060586000F30C8005829C701C8010F
:1002B000F030831605058500F03083120505CF0068
:1002C0000F3048054F0485000800403083160313A3
:1002D00006048600403083120605CE00C601403079
:1002E0004E020319C60A8030831606048600803049
:1002F00083120605CE00CD0180304E020319CD0ACF
:100300004603031D8B29490AC900FF30CE00102087
:10031000F530CE0010204908013A03199629033A16
:100320000319A529013A0319B92908004D03031D32
:10033000080018304B020318A3296430CE001020A7
:100340004B0ACB000800CB0108004D03031D080039
:100350003C304A020318B2296430CE0010204A0A09
:10036000CA0008006430CE0010204B0ACB00CA013E
:100370000800C901CC0108000730831203139F0055
:10038000C030831681008312C701CC01CA01BB01B2
:10039000BC01B901BA01CB01C9010B1712109210AF
:1003A000121507301205CE0018304E049200F930B5
:1003B000831692008B178C1481120116F030010500
:1003C0008312CE0008304E04831681008B178B16E3
:1003D0006521E829D53083120313A000C430A100A1
:1003E000BB30A200DC30A300A401A501A601A70137
:1003F000A801A901AA01AB01AC01AD01AE01AF0199
:10040000C001C101B701B801C201C301C401C501E6
:10041000B001B101B201B301BE01BF01BD018A113A
:100420000A12BC29831203138C1C1B2A83168C1CF2
:100430001B2A3E208C100B1D212A8B1E212A67208F
:100440000B118312360E8400350E8A00340E8300A1
:06045000FF0E7F0E090003
:02400E006A3F07
:00000001FF
